:100000000C9438000C9453000C9453000C9453003F
:100010000C9453000C9453000C9463140C945300F0
:100020000C9453000C9453000C9436140C9453000D
:100030000C942F130C9453000C9453000C94530005
:100040000C9453000C9488030C9453000C945300AC
:100050000C942D110C9453000C9453000C945300E9
:100060000C9453000C9453000C9453000C945300C4
:1000700011241FBECFEFD4E0DEBFCDBF11E0A0E062
:10008000B1E0E8EEFAE202C005900D92A238B107A5
:10009000D9F712E0A2E8B1E001C01D92A239B10780
:1000A000E1F70C9476000C940000CF93DF93CDB76A
:1000B000DEB7E1E3F0E080E18083E4E3F0E08FEF9E
:1000C0008083EAE3F0E08EE28083ABE3B0E0EBE331
:1000D000F0E0808182608C93ABE3B0E0EBE3F0E092
:1000E000808180628C93DF91CF910895CF93DF93CD
:1000F000CDB7DEB723970FB6F894DEBF0FBECDBFE6
:100100000E9455000E9465030E94600F7894A5E349
:10011000B0E0E5E3F0E0808181608C930E943C03D5
:100120000E9446060E9459050E94C4040E942E04A3
:1001300000C0809184018130C9F4109284018981CA
:100140008F5F89830E949B0F198280919101882380
:1001500019F40E94E21306C080910101823014F06C
:100160000E94E2130E940D130E941C1380919301C0
:10017000813079F480919101882319F40E94550609
:1001800006C080910101823014F00E945506109241
:10019000930180919901813069F5A5E3B0E0E5E331
:1001A000F0E0808184608C930E946C0E80919101BC
:1001B000882349F40E948B090E94BF0A0E94760896
:1001C0000E94D90710C080910101823024F00E9462
:1001D00076080E94D90780910101833024F00E94A3
:1001E0008B090E94BF0AA5E3B0E0E5E3F0E080815F
:1001F0008B7F8C9380918201813071F51092820106
:1002000080919101882319F40E942E0406C08091E8
:100210000101833014F00E942E0480918E01909190
:100220008F01019690938F0180938E0180918E01B2
:1002300090918F018C33910569F480918C0190919C
:100240008D01019690938D0180938C0110928F0106
:1002500010928E010E94680580918301813009F01F
:1002600068CF109283010E94BF118091910181306B
:1002700009F05FCF80919001813009F05ACF109240
:10028000900180910101282F332727FD30953B8372
:100290002A838A819B8181309105C1F02A813B812B
:1002A000223031052CF48A819B81009761F041CF87
:1002B0002A813B812230310571F08A819B81833014
:1002C0009105B1F036CF0E94180433CF0E94230469
:1002D0000E94910C2ECF0E94230464E084E00E94CF
:1002E000A4010E9446060E9459050E94C40421CF21
:1002F0000E94230464E084E00E94A4010E94460658
:100300000E9459050E94C4040E942E0412CFCF936C
:10031000DF93CDB7DEB764E084E00E94A4016CE413
:1003200080E00E94A40110928401809184018823BE
:10033000E1F36AE08CE60E94A40160E085E00E949F
:10034000A401DF91CF910895CF93DF93CDB7DEB7AE
:1003500024970FB6F894DEBF0FBECDBF8B836C839E
:10036000ABE3B0E0EBE3F0E080818D7F8C9387E03E
:100370008A8340C0ABE3B0E0EBE3F0E08081877FAD
:100380008C9300000000000000008A81282F332792
:1003900027FD309581E090E0022E02C0880F991F62
:1003A0000A94E2F7982F8B81892389838981882396
:1003B00041F0ABE3B0E0EBE3F0E0808184608C934C
:1003C00007C0ABE3B0E0EBE3F0E080818B7F8C9380
:1003D0000000000000000000ABE3B0E0EBE3F0E061
:1003E000808188608C9300000000000000008A81FA
:1003F00081508A838A8188230CF0BCCF87E08A836E
:1004000040C0ABE3B0E0EBE3F0E08081877F8C930A
:1004100000000000000000008A81282F332727FDFC
:10042000309581E090E0022E02C0880F991F0A9457
:10043000E2F7982F8C81892389838981882341F071
:10044000ABE3B0E0EBE3F0E0808184608C9307C025
:10045000ABE3B0E0EBE3F0E080818B7F8C930000B6
:10046000000000000000ABE3B0E0EBE3F0E08081CF
:1004700088608C9300000000000000008A81815099
:100480008A838A8188230CF0BCCFABE3B0E0EBE336
:10049000F0E08081877F8C93ABE3B0E0EBE3F0E0AA
:1004A00080818B7F8C93ABE3B0E0EBE3F0E0808165
:1004B00082608C9324960FB6F894DEBF0FBECDBF3A
:1004C000DF91CF910895CF93DF93CDB7DEB7249717
:1004D0000FB6F894DEBF0FBECDBF8C83ABE3B0E0A8
:1004E000EBE3F0E080818D7F8C9387E08A834CC0C2
:1004F000ABE3B0E0EBE3F0E08081877F8C9300001A
:1005000000000000000000000000000000008A81E0
:10051000282F332727FD309581E090E0022E02C07E
:10052000880F991F0A94E2F7982F8C8189238B8377
:100530008B81181644F4ABE3B0E0EBE3F0E080818C
:1005400084608C9307C0ABE3B0E0EBE3F0E0808124
:100550008B7F8C9300000000000000000000000072
:1005600000000000ABE3B0E0EBE3F0E080818860E6
:100570008C9300000000000000000000000000005C
:1005800000008A8181508A838A8188230CF0B0CF51
:100590001B82ABE3B0E0EBE3F0E08081877F8C93DC
:1005A000000000000000000000000000000000004B
:1005B00087E08A833DC0ABE3B0E0EBE3F0E080810D
:1005C00088608C93E9E3F0E08081898389819927B1
:1005D00080719070181619068CF48A81282F3327A1
:1005E00027FD309581E090E0022E02C0880F991F10
:1005F0000A94E2F7982F8B81892B8B8300000000EF
:10060000000000000000000000000000ABE3B0E0CC
:10061000EBE3F0E08081877F8C9300000000000016
:10062000000000000000000000008A8181508A83E1
:100630008A8188230CF0BFCFABE3B0E0EBE3F0E0BE
:100640008081877F8C93ABE3B0E0EBE3F0E08081C7
:100650008B7F8C93ABE3B0E0EBE3F0E080818260D2
:100660008C938B81992724960FB6F894DEBF0FBE2A
:10067000CDBFDF91CF910895CF93DF93CDB7DEB794
:100680000E94870110928201809182018823E1F308
:100690000E946B040E94910C109282018091820151
:1006A0008823E1F310928201809182018823E1F393
:1006B0001092820164E084E00E94A4016CE480E076
:1006C0000E94A401DF91CF910895CF93DF93CDB71E
:1006D000DEB7E3E5F0E082E08083EEE4F0E082E480
:1006E0008083E9E5F0E08AE18083E7E4F0E086E0FA
:1006F0008083E2E4F0E080EF8083EAE8F0E083E4E6
:100700008083EDE7F0E080E28083DF91CF91089570
:100710001F920F920FB60F9211248F93CF93DF93F6
:10072000CDB7DEB7809186018F5F8093860180917F
:100730008601883459F581E0809385011092860105
:1007400080914D028F5F80934D0280914D028436DF
:1007500041F410924D0281E08093820181E0809308
:10076000830180914D02823319F481E080938301EB
:1007700080914C028F5F80934C0280914C028A30B2
:1007800029F410924C0281E080938401DF91CF9193
:100790008F910F900FBE0F901F901895CF93DF93FE
:1007A000CDB7DEB762E480E00E94A401109282011E
:1007B000809182018823E1F3109282016BE689E047
:1007C0000E94A40110928401809184018823E1F3A6
:1007D0001092840110924E0216C080914E02682F32
:1007E0008AE00E94A40180914E029927FC01E95CF5
:1007F000FE4F8081682F8BE00E94A40180914E0201
:100800008F5F80934E0280914E02863330F360EA10
:1008100088E00E94A40110928401809184018823C1
:10082000E1F36CE480E00E94A401DF91CF91089590
:10083000CF93DF93CDB7DEB762E480E00E94A401DE
:10084000DF91CF910895CF93DF93CDB7DEB76CE4FE
:1008500080E00E94A401DF91CF910895CF93DF93B0
:10086000CDB7DEB789ED80934E0213C060E085E01E
:100870000E94A40180914E02682F86E00E94A4018C
:1008800064E587E00E94A40180914E028F5F80930F
:100890004E0280914E028C3D48F385EE80934E02CD
:1008A00013C060E085E00E94A40180914E02682F91
:1008B00086E00E94A40164E587E00E94A401809183
:1008C0004E028F5F80934E0280914E02883E48F325
:1008D000DF91CF910895CF93DF93CDB7DEB76497C3
:1008E0000FB6F894DEBF0FBECDBF8DE589838EE5D0
:1008F0008A838FE58B8389E48C838BE58D838DE1FF
:100900008E838CE58F83188680E2898789E28A87C7
:1009100086E38B8781E48C878AE08D8781E48E87EC
:1009200085E08F8786E2888B20E1CE010196AC01BD
:1009300062E087E00E94EF0464960FB6F894DEBF91
:100940000FBECDBFDF91CF910895CF93DF93CDB789
:10095000DEB760E085E00E94A4016FEC86E00E94B3
:10096000A4016CE887E00E94A40161E085E00E9498
:10097000A4016BE086E00E94A4016DE887E00E947C
:10098000A401DF91CF910895CF93DF93CDB7DEB768
:1009900060E085E00E94A40160E286E00E94A4017C
:1009A00060E887E00E94A40160E085E00E94A40165
:1009B0006EE386E00E94A40164E887E00E94A4013F
:1009C00060E085E00E94A4016CE586E00E94A4013D
:1009D00068E887E00E94A401DF91CF910895CF934A
:1009E000DF93CDB7DEB72D970FB6F894DEBF0FBEFD
:1009F000CDBF89876A875C874B872D878A85282F9B
:100A000033278EE190E0A901489F9001499F300D66
:100A1000589F300D112489859927820F931F98873D
:100A20008F838D85282F33278F819885820F931F81
:100A30009E838D8310924E028F8198859C838B8339
:100A400028C08B818A838B819C81892F99278983F8
:100A5000698185E00E94A4016A8186E00E94A40168
:100A600040914E02842F99279C018B859C85F9012A
:100A7000E80FF91F8081982F842F8F5F80934E029B
:100A8000692F87E00E94A4018B819C8101969C8341
:100A90008B832B813C818D819E812817390788F2B9
:100AA0002D960FB6F894DEBF0FBECDBFDF91CF916C
:100AB0000895CF93DF93CDB7DEB786E091E025E0D0
:100AC000AC016EE087E10E94EF04DF91CF910895C1
:100AD0000F931F93CF93DF93CDB7DEB729970FB650
:100AE000F894DEBF0FBECDBF18868AE089872091BB
:100AF0008C0130918D01CE0102964AE050E0BC019C
:100B0000C9010E941C15CE010296DC01FD01019075
:100B10000020E9F73197CF018A1B9B0B8983109244
:100B20004E021CC080914E02082F112780914E0268
:100B3000282F3327CE010296FC01E20FF31F80819C
:100B40000E94E206282FCE010596FC01E00FF11F5E
:100B5000208380914E028F5F80934E0280914E02DF
:100B6000282F33278981992787FD909528173907E2
:100B7000CCF280918C0190918D018A3091058CF49A
:100B8000CE01089621E0AC016EE087E10E94EF04FF
:100B9000CE01059621E0AC016EE088E10E94EF04F1
:100BA00008C0CE01059622E0AC016EE087E10E940C
:100BB000EF0420918E0130918F01CE0102964AE020
:100BC00050E0BC01C9010E941C15CE010296DC0157
:100BD000FD0101900020E9F73197CF018A1B9B0BA3
:100BE000898310924E021CC080914E02082F11275B
:100BF00080914E02282F3327CE010296FC01E20F8E
:100C0000F31F80810E94E206282FCE010596FC0189
:100C1000E00FF11F208380914E028F5F80934E0280
:100C200080914E02282F33278981992787FD90953F
:100C300028173907CCF280918E0190918F018A306C
:100C400091058CF4CE01099621E0AC016EE08AE1B9
:100C50000E94EF04CE01059621E0AC016EE08BE12D
:100C60000E94EF0408C0CE01059622E0AC016EE0C0
:100C70008AE10E94EF0429960FB6F894DEBF0FBEFA
:100C8000CDBFDF91CF911F910F910895CF93DF9347
:100C9000CDB7DEB782E091E024E0AC016EE082E007
:100CA0000E94EF04DF91CF9108950F931F93CF938C
:100CB000DF93CDB7DEB761970FB6F894DEBF0FBEF6
:100CC000CDBFCE010A969E878D87E7E7F1E0F88BCE
:100CD000EF87F3E0F98BEF85F88900808F8598899D
:100CE0000196988B8F87ED85FE8500828D859E8588
:100CF00001969E878D8799899150998BE989EE237A
:100D000051F72091AF013091B001CE0102964AE037
:100D100050E0BC01C9010E941C15CE010296DC0105
:100D2000FD0101900020E9F73197CF018A1B9B0B51
:100D3000898310924E021CC080914E02082F112709
:100D400080914E02282F3327CE010296FC01E20F3C
:100D5000F31F80810E94E206282FCE010696FC0137
:100D6000E00FF11F208380914E028F5F80934E022F
:100D700080914E02282F33278981992787FD9095EE
:100D800028173907CCF2CE010A9623E0AC016DE0BA
:100D90008DE00E94EF042981998180E1382F391B71
:100DA000CE010696AC016DE0832F0E94EF046196A0
:100DB0000FB6F894DEBF0FBECDBFDF91CF911F916C
:100DC0000F910895CF93DF93CDB7DEB722970FB67B
:100DD000F894DEBF0FBECDBF8A838A818D3219F4AD
:100DE00089E4898309C08A81803319F48AE0898380
:100DF00003C08A81805389838981992787FD9095D3
:100E000022960FB6F894DEBF0FBECDBFDF91CF9113
:100E100008950F931F93CF93DF93CDB7DEB76097FD
:100E20000FB6F894DEBF0FBECDBF85E0FE013C9645
:100E3000DF01982F1D929A95E9F72091AD0130912D
:100E4000AE01CE0102964AE050E0BC01C9010E9409
:100E50001C15CE010296DC01FD0101900020E9F78E
:100E60003197CF018A1B9B0B898310924E021CC0C5
:100E700080914E02082F112780914E02282F332790
:100E8000CE010296FC01E20FF31F80810E94E20670
:100E9000282FCE010796FC01E00FF11F20838091DF
:100EA0004E028F5F80934E0280914E02282F33278F
:100EB0008981992787FD909528173907CCF2CE01B3
:100EC0000C9624E0AC0167E089E10E94EF042981DF
:100ED00099818CE1382F391BCE010796AC0167E070
:100EE000832F0E94EF048091AD019091AE011816FE
:100EF0001906C4F460E085E00E94A4016FEC86E06E
:100F00000E94A4016CE887E00E94A40161E085E0F2
:100F10000E94A4016BE086E00E94A40160E087E0EB
:100F20000E94A4018091AD019091AE019923C4F477
:100F300060E085E00E94A4016FEC86E00E94A401BD
:100F400060E087E00E94A40161E085E00E94A401C6
:100F50006BE086E00E94A4016DE887E00E94A40196
:100F60008091AD019091AE010097C1F460E085E001
:100F70000E94A4016FEC86E00E94A40160E087E07B
:100F80000E94A40161E085E00E94A4016BE086E07C
:100F90000E94A40160E087E00E94A40160960FB661
:100FA000F894DEBF0FBECDBFDF91CF911F910F919F
:100FB00008950F931F93CF93DF93CDB7DEB7659757
:100FC0000FB6F894DEBF0FBECDBFCE010E969A8B42
:100FD000898BEAE7F1E0FC8BEB8BF3E0FD8BEB898F
:100FE000FC8900808B899C8901969C8B8B8BE9897D
:100FF000FA89008289899A8901969A8B898B9D89C1
:1010000091509D8BED89EE2351F780915B02909179
:101010005C022EE130E0B9010E946115CB019B8397
:101020008A838A819B81992314F41B821A82CE01C0
:1010300004962A813B814AE050E0BC01C9010E942C
:101040001C15CE010496DC01FD0101900020E9F79A
:101050003197CF018A1B9B0B898310924E021CC0D3
:1010600080914E02082F112780914E02282F33279E
:10107000CE010496FC01E20FF31F80810E94E2067C
:10108000282FCE010996FC01E00FF11F20838091EB
:101090004E028F5F80934E0280914E02282F33279D
:1010A0008981992787FD909528173907CCF2CE01C1
:1010B0000E9623E0AC016EE081E00E94EF042981EE
:1010C000998184E0382F391BCE010996AC016EE07E
:1010D000832F0E94EF0465960FB6F894DEBF0FBE13
:1010E000CDBFDF91CF911F910F910895CF93DF93E3
:1010F000CDB7DEB729970FB6F894DEBF0FBECDBFD0
:1011000080916302909164028E5590409C838B8302
:101110008B819C8123E030E0B9010E946115CB01F5
:101120009A83898389819A818A30910524F089E0A4
:1011300090E09A83898389819A81992314F41A8291
:10114000198220918A0130918B0189819A818217BD
:10115000930709F4D7C089819A81823091052CF4D4
:1011600060E184E00E94A40104C060E084E00E9489
:10117000A40189819A8190938B0180938A0180E8F0
:101180008D8384E88E8388E88F8389819A8199870B
:101190008887888599858430910509F45FC08885A2
:1011A000998585309105DCF4888599858130910594
:1011B00009F43FC088859985823091052CF4888593
:1011C0009985009779F173C088859985823091055A
:1011D000B9F18885998583309105C9F168C0888502
:1011E00099858730910509F44EC0888599858830A6
:1011F00091055CF48885998585309105B1F18885E4
:10120000998586309105C1F152C0888599858830CD
:10121000910509F43FC0888599858930910509F4C5
:1012200040C045C080E88D8384E88E8388E88F8342
:101230003EC081E88D8384E88E8388E88F8337C041
:1012400082E88D8384E88E8388E88F8330C083E8CA
:101250008D8384E88E8388E88F8329C083E88D831B
:1012600085E88E8388E88F8322C083E88D8386E8B3
:101270008E8388E88F831BC083E88D8387E88E8305
:1012800088E88F8314C083E88D8387E88E8389E89C
:101290008F830DC083E88D8387E88E838AE88F83F0
:1012A00006C083E88D8387E88E838BE88F8360E0B8
:1012B00085E00E94A40160E286E00E94A4018D8185
:1012C000682F87E00E94A40160E085E00E94A401ED
:1012D0006EE386E00E94A4018E81682F87E00E9461
:1012E000A40160E085E00E94A4016CE586E00E9414
:1012F000A4018F81682F87E00E94A40160E084E050
:101300000E94A40129960FB6F894DEBF0FBECDBF90
:10131000DF91CF910895CF93DF93CDB7DEB72697B6
:101320000FB6F894DEBF0FBECDBF809153029091EF
:10133000540226E130E0B9010E946115CB01069606
:101340009E838D838D819E8199230CF446C08D816F
:101350009E812AE030E0B9010E946115CB018A83A9
:101360008D819E812AE030E0B9010E946115898358
:10137000898186958C5F89838A81282F332786E827
:1013800090E0821B930B9C838B8320910D01309105
:101390000E018B819C818217930761F080910D0172
:1013A00090910E010E94440A8B819C8169810E9468
:1013B0007E0A0AC0909197018981981729F08B8144
:1013C0009C8169810E947E0A8981809397018B812B
:1013D0009C8190930E0180930D018D819E819923B4
:1013E0000CF049C08D819E81909581959F4F9E8381
:1013F0008D838D819E812AE030E0B9010E946115C4
:10140000CB018A838D819E812AE030E0B9010E9460
:10141000611589838981869589838A8199278A576D
:101420009F4F9C838B8320910D0130910E018B8106
:101430009C818217930761F080910D0190910E01BC
:101440000E94440A8B819C8169810E947E0A0AC0A5
:10145000909197018981981729F08B819C816981EE
:101460000E947E0A8981809397018B819C81909351
:101470000E0180930D0126960FB6F894DEBF0FBEC5
:10148000CDBFDF91CF910895CF93DF93CDB7DEB776
:1014900026970FB6F894DEBF0FBECDBF9E838D8317
:1014A0001C821B821DC08D818A838D819E81892F24
:1014B00099278983698185E00E94A4016A8186E079
:1014C0000E94A40160E087E00E94A4018D819E81BA
:1014D0004E969E838D838B819C8101969C838B830A
:1014E0008B819C8188309105F0F226960FB6F89496
:1014F000DEBF0FBECDBFDF91CF910895CF93DF93B5
:10150000CDB7DEB727970FB6F894DEBF0FBECDBFBD
:101510009E838D836F831C821B8223C08D818A836F
:101520008D819E81892F99278983698185E00E9419
:10153000A4016A8186E00E94A4018F819927FC01A1
:10154000E35DFE4F8081682F87E00E94A4018D81BA
:101550009E814E969E838D838B819C8101969C8378
:101560008B838B819C8188309105C0F227960FB6C2
:10157000F894DEBF0FBECDBFDF91CF910895CF931A
:10158000DF93CDB7DEB726970FB6F894DEBF0FBE58
:10159000CDBF809151029091520226E130E0B90115
:1015A0000E946115CB019E838D838D819E8199233D
:1015B0000CF452C08D819E812AE030E0B9010E9476
:1015C0006115CB018A838D819E812AE030E0B901CB
:1015D0000E94611589838981869589838A81282F54
:1015E000332787E090E0AC01421B530B9A018EE158
:1015F00090E0AC01249FC001259F900D349F900D79
:1016000011240A969C838B8320910B0130910C014D
:101610008B819C818217930761F080910B019091DF
:101620000C010E948F0B8B819C8169810E94F20BBF
:101630000AC0909196018981981729F08B819C812D
:1016400069810E94F20B8981809396018B819C8134
:1016500090930C0180930B018D819E8199230CF056
:1016600055C08D819E81909581959F4F9E838D83DE
:101670008D819E812AE030E0B9010E946115CB0185
:101680008A838D819E812AE030E0B9010E94611534
:101690008983898186958C5F89838A81282F332766
:1016A0008EE190E0AC01249FC001259F900D349FF6
:1016B000900D112486509F4F9C838B8320910B01AA
:1016C00030910C018B819C818217930761F080918E
:1016D0000B0190910C010E948F0B8B819C81698181
:1016E0000E94F20B0AC0909196018981981729F007
:1016F0008B819C8169810E94F20B89818093960184
:101700008B819C8190930C0180930B0126960FB6E0
:10171000F894DEBF0FBECDBFDF91CF910895CF9378
:10172000DF93CDB7DEB726970FB6F894DEBF0FBEB6
:10173000CDBF9E838D838D819E819C838B8318C0BA
:101740008B818A838B819C81892F992789836981E9
:1017500085E00E94A4016A8186E00E94A40160E005
:1017600087E00E94A4018B819C8101969C838B83DE
:101770008D819E819C01275F3F4F8B819C818217C9
:101780009307F0F280919601282F3327C901880F23
:10179000991F820F931FFC01EF5EFE4F808188230B
:1017A000C1F08D819E8182969C838B838B818A83FD
:1017B0008B819C81892F99278983698185E00E948B
:1017C000A4016A8186E00E94A40160E087E00E9493
:1017D000A40126960FB6F894DEBF0FBECDBFDF91F1
:1017E000CF910895CF93DF93CDB7DEB727970FB68C
:1017F000F894DEBF0FBECDBF9E838D836F838D8136
:101800009E819C838B8324C08B8189838B819C8167
:10181000892F99278A836A8185E00E94A4016981C2
:1018200086E00E94A4018F81282F3327C901880FE9
:10183000991F820F931FFC01E15FFE4F8081682F8B
:1018400087E00E94A4018B819C8101969C838B83FD
:101850008D819E819C01275F3F4F8B819C818217E8
:10186000930790F28D819E8104969C838B838B815C
:1018700089838B819C81892F99278A836A8185E05E
:101880000E94A401698186E00E94A4018F81282F13
:101890003327C901880F991F820F931FFC01E05F56
:1018A000FE4F8081682F87E00E94A4018F81282F3E
:1018B0003327C901880F991F820F931FFC01EF5E28
:1018C000FE4F8081882321F18D819E8182969C83A9
:1018D0008B838B8189838B819C81892F99278A8334
:1018E0006A8185E00E94A401698186E00E94A401CA
:1018F0008F81282F3327C901880F991F820F931FCB
:10190000FC01EF5EFE4F8081682F87E00E94A401FA
:1019100027960FB6F894DEBF0FBECDBFDF91CF91F3
:101920000895CF93DF93CDB7DEB760E085E00E94E6
:10193000A40163E886E00E94A40160E987E00E94B8
:10194000A40160E085E00E94A40164E886E00E94B2
:10195000A40161E987E00E94A40160E085E00E94A3
:10196000A40165E886E00E94A40162E987E00E9484
:10197000A40160E085E00E94A40166E886E00E9480
:10198000A40163E987E00E94A40160E085E00E9471
:10199000A40167E886E00E94A40164E987E00E9450
:1019A000A40160E085E00E94A40168E886E00E944E
:1019B000A40165E987E00E94A40160E085E00E943F
:1019C000A40169E886E00E94A40166E987E00E941C
:1019D000A40160E085E00E94A4016AE886E00E941C
:1019E000A40167E987E00E94A40160E085E00E940D
:1019F000A40161EA86E00E94A40168E987E00E94F0
:101A0000A40160E085E00E94A40162EA86E00E94F1
:101A1000A40169E987E00E94A40160E085E00E94DA
:101A2000A40163EA86E00E94A4016AE987E00E94BB
:101A3000A40160E085E00E94A40164EA86E00E94BF
:101A4000A4016BE987E00E94A40160E085E00E94A8
:101A5000A40165EA86E00E94A4016CE987E00E9487
:101A6000A40160E085E00E94A40166EA86E00E948D
:101A7000A4016DE987E00E94A40160E085E00E9476
:101A8000A40167EA86E00E94A4016EE987E00E9453
:101A9000A40160E085E00E94A40168EA86E00E945B
:101AA000A4016FE987E00E94A40160E085E00E9444
:101AB000A4016FEB86E00E94A40160EA87E00E9427
:101AC000A40160E085E00E94A40160EC86E00E9431
:101AD000A40161EA87E00E94A40160E085E00E9421
:101AE000A40161EC86E00E94A40162EA87E00E9402
:101AF000A40160E085E00E94A40162EC86E00E94FF
:101B0000A40163EA87E00E94A40160E085E00E94EE
:101B1000A40163EC86E00E94A40164EA87E00E94CD
:101B2000A40160E085E00E94A40164EC86E00E94CC
:101B3000A40165EA87E00E94A40160E085E00E94BC
:101B4000A40165EC86E00E94A40166EA87E00E9499
:101B5000A40160E085E00E94A40166EC86E00E949A
:101B6000A40167EA87E00E94A40160E085E00E948A
:101B7000A4016DED86E00E94A40168EA87E00E945E
:101B8000A40160E085E00E94A4016EED86E00E9461
:101B9000A40169EA87E00E94A40160E085E00E9458
:101BA000A4016FED86E00E94A4016AEA87E00E942A
:101BB000A40160E085E00E94A40160EE86E00E943E
:101BC000A4016BEA87E00E94A40160E085E00E9426
:101BD000A40161EE86E00E94A4016CEA87E00E9405
:101BE000A40160E085E00E94A40162EE86E00E940C
:101BF000A4016DEA87E00E94A40160E085E00E94F4
:101C0000A40163EE86E00E94A4016EEA87E00E94D0
:101C1000A40160E085E00E94A40164EE86E00E94D9
:101C2000A4016FEA87E00E94A40160E085E00E94C1
:101C3000A4016BEF86E00E94A40160EB87E00E94A4
:101C4000A40160E085E00E94A4016CEF86E00E94A0
:101C5000A40161EB87E00E94A40160E085E00E949E
:101C6000A4016DEF86E00E94A40162EB87E00E9470
:101C7000A40160E085E00E94A4016EEF86E00E946E
:101C8000A40163EB87E00E94A40160E085E00E946C
:101C9000A4016FEF86E00E94A40164EB87E00E943C
:101CA000A40161E085E00E94A40160E086E00E945A
:101CB000A40165EB87E00E94A40161E085E00E9439
:101CC000A40161E086E00E94A40166EB87E00E9427
:101CD000A401DF91CF910895CF93DF93CDB7DEB705
:101CE00064970FB6F894DEBF0FBECDBF83E090E0DF
:101CF0009C8B8B8B1A82198283E990E09C838B8367
:101D0000CFC08B899C89FC01EF54FE4F80819927BD
:101D1000CD979A8B898B8B899C8901969C8B8B8B19
:101D20008B899C89FC01EF54FE4F80819927CD97C8
:101D3000988B8F878B899C8901969C8B8B8B8B8949
:101D40009C89FC01EF54FE4F80819927CD979E8797
:101D50008D878B899C8901969C8B8B8B8B899C8929
:101D6000FC01EF54FE4F80819927CD979C878B878C
:101D70008B899C8901969C8B8B8B89899A899C0184
:101D8000220F331F220F331F8F85988995958795D2
:101D9000959587959595879595958795822B932B06
:101DA0009A8789878F8598898F7090709C0122957A
:101DB0003295307F3227207F32278D859E859595FD
:101DC000879595958795822B932B98878F838D8503
:101DD0009E85837090709C0100243695279507940A
:101DE000369527950794322F202D8B859C85822B45
:101DF000932B9E838D838B819C8101979C838B8306
:101E00008B819C812FEF8F3F920709F44EC089810F
:101E10009A819C0180917D0190917E01F901E80FEA
:101E2000F91F8985808389819A8101969A838983A4
:101E30008B819C8101979C838B838B819C812FEF6D
:101E40008F3F920791F189819A819C0180917D0158
:101E500090917E01F901E80FF91F8F8180838981BC
:101E60009A8101969A8389838B819C8101979C83B7
:101E70008B838B819C812FEF8F3F9207B1F08981FB
:101E80009A819C0180917D0190917E01F901E80F7A
:101E9000F91F8D81808389819A8101969A83898334
:101EA0008B819C81009709F02CCF10929901649648
:101EB0000FB6F894DEBF0FBECDBFDF91CF9108956E
:101EC000CF93DF93CDB7DEB7E9E2F0E082E2808323
:101ED000E0E4F0E01082E0E2F0E082E28083ECE512
:101EE000F0E01082A2E3B0E0E2E3F0E08081816004
:101EF0008C93A8E3B0E0E8E3F0E0808184608C9309
:101F0000EAE2F0E088E98083E0E4F0E086E88083BC
:101F1000EBE2F0E082EC8083E1E2F0E088E98083AC
:101F2000ECE5F0E086E88083E2E2F0E082EC80839A
:101F3000DF91CF910895CF93DF93CDB7DEB764974C
:101F40000FB6F894DEBF0FBECDBF83E28F83188635
:101F500083E689871A861B8685E090E09E838D83C1
:101F60001C821B821A82198215C029813A81CE01F6
:101F70000796FC01E20FF31F8081282F33278B8106
:101F80009C81820F931F9C838B8389819A81019608
:101F90009A83898329813A818D819E812817390707
:101FA00024F38B819C8120E030E1B9010E9461150E
:101FB0009C838B838D819E819A8B898B8B819C8165
:101FC0009C8B8B8B8B899C8999232CF48B899C8986
:101FD000CF969C8B8B8B8B899C89082E892F000C2C
:101FE000881F990B000C881F991F282F235CCE0196
:101FF0000796E989FA89E80FF91F20838D819E8170
:1020000001969E838D83ED81FE818B819C8120E4EE
:1020100030E0B9010E946115282F235CCE0107969C
:10202000E80FF91F20838D819E8101969E838D8309
:102030002D813E81CE010796FC01E20FF31F8DE05A
:1020400080838D819E8101969E838D831A82198261
:102050000FC029813A81CE010796FC01E20FF31FE0
:1020600080810E94461089819A8101969A83898392
:1020700089819A818830910564F364960FB6F8944B
:10208000DEBF0FBECDBFDF91CF910895CF93DF9319
:10209000CDB7DEB721970FB6F894DEBF0FBECDBF28
:1020A0008983E2E2F0E08081992780729070009746
:1020B000C1F3E3E2F0E08981808321960FB6F894C2
:1020C000DEBF0FBECDBFDF91CF910895CF93DF93D9
:1020D000CDB7DEB721970FB6F894DEBF0FBECDBFE8
:1020E0008983EBE2F0E080819927807290700097FD
:1020F000C1F3ECE2F0E08981808321960FB6F89479
:10210000DEBF0FBECDBFDF91CF910895CF93DF9398
:10211000CDB7DEB726970FB6F894DEBF0FBECDBFA2
:102120009E838D838D819E81DC01FD0101900020C5
:10213000E9F73197CF018A1B9B0B9C838B831A8213
:1021400019820FC029813A818D819E81F901E80FA2
:10215000F91F80810E94661089819A8101969A8375
:10216000898329813A818B819C818217930750F75B
:1021700080917F010E946610809180010E9466100C
:1021800026960FB6F894DEBF0FBECDBFDF91CF917C
:102190000895CF93DF93CDB7DEB72C970FB6F894A1
:1021A000DEBF0FBECDBF9C878B878B859C854AE0A9
:1021B00050E09E012F5F3F4FB9010E941C15CE01D8
:1021C00001960E9486102C960FB6F894DEBF0FBEC3
:1021D000CDBFDF91CF910895CF93DF93CDB7DEB719
:1021E00022970FB6F894DEBF0FBECDBF8A8387E07B
:1021F00089831FC08A81482F55278981282F33273B
:1022000027FD309581E090E0022E02C0880F991FD3
:102210000A94E2F7842395231816190624F481E31F
:102220000E94661003C080E30E946610898181507D
:10223000898389818823F4F680917F010E9466104A
:10224000809180010E94661022960FB6F894DEBF3E
:102250000FBECDBFDF91CF9108951F920F920FB6A1
:102260000F9211242F933F938F939F93AF93BF931C
:10227000EF93FF93CF93DF93CDB7DEB72297DEBF07
:10228000CDBFE3E2F0E080818093910280919102E2
:102290008D30D1F4809198018130B1F4A5E3B0E0A4
:1022A000E5E3F0E08081877F8C931092980181E0D4
:1022B0008093990180914902992720919102FC0114
:1022C000EF54FE4F208348C080919801282F332778
:1022D0003A83298389819A81009731F029813A8153
:1022E0002130310521F138C080919102833271F49F
:1022F00080919901882351F481E080939801A5E3AE
:10230000B0E0E5E3F0E0808188608C9310924902B0
:1023100030914902832F992720919102FC01EF54BB
:10232000FE4F2083832F8F5F8093490215C08091D9
:102330004902992720919102FC01EF54FE4F20831E
:1023400080914902863930F4809149028F5F8093F1
:10235000490202C0109298012296F894DEBFCDBFC8
:10236000DF91CF91FF91EF91BF91AF919F918F91AD
:102370003F912F910F900FBE0F901F901895CF9304
:10238000DF93CDB7DEB76E970FB6F894DEBF0FBE02
:10239000CDBF2091510230915202CE010B964AE0FE
:1023A00050E0BC01C9010E941C1580E4898384E4CB
:1023B0008A8380E38B831C82CE010B96DC01FD01B6
:1023C00001900020E9F73197CF018A1B9B0B9E01FA
:1023D000255F3F4FAC01B901CE0101960E940C155B
:1023E000CE010196DC01FD0101900020E9F7319753
:1023F0009F012A1B3B0BCE010196820F931FFC010C
:1024000083E290E091838083CE0101960E94861042
:102410002091530230915402CE010B964AE050E0D5
:10242000BC01C9010E941C1580E4898384E48A836D
:1024300081E38B831C82CE010B96DC01FD010190B0
:102440000020E9F73197CF018A1B9B0B9E01255F86
:102450003F4FAC01B901CE0101960E940C15CE018F
:102460000196DC01FD0101900020E9F731979F0101
:102470002A1B3B0BCE010196820F931FFC0183E2C6
:1024800090E091838083CE0101960E948610209176
:102490005B0230915C02CE010B964AE050E0BC0139
:1024A000C9010E941C1580E4898388E68A838DE334
:1024B0008B831C82CE010B96DC01FD010190002074
:1024C000E9F73197CF018A1B9B0B9E01255F3F4F98
:1024D000AC01B901CE0101960E940C15CE01019606
:1024E000DC01FD0101900020E9F731979F012A1BD3
:1024F0003B0BCE010196820F931FFC0183E290E01B
:1025000091838083CE0101960E9486102091630200
:1025100030916402CE010B964AE050E0BC01C90143
:102520000E941C1580E4898386E58A838CE68B8370
:102530001C82CE010B96DC01FD0101900020E9F721
:102540003197CF018A1B9B0B9E01255F3F4FAC014A
:10255000B901CE0101960E940C15CE010196DC0155
:10256000FD0101900020E9F731979F012A1B3B0BE9
:10257000CE010196820F931FFC0183E290E09183CC
:102580008083CE0101960E9486102091AF01309188
:10259000B001CE010B964AE050E0BC01C9010E9497
:1025A0001C1580E489838BE48A8387E68B831C82F5
:1025B000CE010B96DC01FD0101900020E9F7319777
:1025C000CF018A1B9B0B9E01255F3F4FAC01B901D8
:1025D000CE0101960E940C15CE010196DC01FD0191
:1025E00001900020E9F731979F012A1B3B0BCE0198
:1025F0000196820F931FFC0183E290E09183808318
:10260000CE0101960E9486106E960FB6F894DEBF3A
:102610000FBECDBFDF91CF910895CF93DF93CDB79C
:10262000DEB7A5E3B0E0E5E3F0E0908182E0892742
:102630008C93DF91CF910895CF93DF93CDB7DEB721
:1026400080918901813041F4A5E3B0E0E5E3F0E059
:10265000908181E089278C93DF91CF9108951F921B
:102660000F920FB60F9211242F933F934F935F93C6
:102670006F937F938F939F93AF93BF93EF93FF934A
:10268000CF93DF93CDB7DEB780919A0190919B01F4
:102690000097B1F4E4E4F0E0808191819093A1018E
:1026A0008093A001AEE4B0E0EEE4F0E080818F7BA7
:1026B0008C9381E090E090939B0180939A016FC08E
:1026C000E4E4F0E08081918190939F0180939E01EA
:1026D000AEE4B0E0EEE4F0E0808180648C93209181
:1026E0009E0130919F018091A0019091A101A901CB
:1026F000481B590BCA0190939D0180939C01109235
:102700009B0110929A0180919C0190919D018656A7
:10271000984090939D0180939C0180919C019091A1
:102720009D012CE231E0B9010E944D15CB0190933F
:102730009D0180939C0180919C0190919D01992322
:1027400024F410929D0110929C0180919C01909123
:102750009D018730910534F086E090E090939D01D3
:1027600080939C0180910101282F332727FD30950C
:1027700080919C0190919D012817390781F08091EB
:102780009C0190919D01863091054CF480919C01B3
:1027900090919D018093010181E080939001DF91F0
:1027A000CF91FF91EF91BF91AF919F918F917F91C9
:1027B0006F915F914F913F912F910F900FBE0F90AE
:1027C0001F901895CF93DF93CDB7DEB780915B0252
:1027D00090915C02909348028093470220914702B7
:1027E000309148028091AB019091AC01A901481B46
:1027F000590BCA019093AA018093A90180914702C5
:10280000909148029093AC018093AB012091A70175
:102810003091A8018091A9019091AA01820F931F84
:102820009093A8018093A701809192018F5F80937C
:102830009201809192018630B1F4109292018091C0
:10284000A7019091A80125E030E0B9010E9461152F
:10285000CB019093AE018093AD011092A80110922C
:10286000A7010E940907DF91CF9108951F920F924F
:102870000FB60F9211248F939F93AF93BF93EF9353
:10288000FF93CF93DF93CDB7DEB7E3E4F0E01082A0
:102890008091AD019091AE01009741F0A2E3B0E0CC
:1028A000E2E3F0E0908188E089278C93DF91CF917B
:1028B000FF91EF91BF91AF919F918F910F900FBEBC
:1028C0000F901F9018951F920F920FB60F92112420
:1028D0002F933F934F935F936F937F938F939F9328
:1028E000AF93BF93EF93FF93CF93DF93CDB7DEB753
:1028F0008091A2018823D1F4E0E8F0E08081918109
:102900009093A4018093A301AAE8B0E0EAE8F0E084
:1029100080818F7B8C9381E08093A201A2E3B0E061
:10292000E2E3F0E0808180618C9363C0E8E8F0E04E
:1029300011821082E0E8F0E0808191819093A601FD
:102940008093A501AAE8B0E0EAE8F0E08081806425
:102950008C931092A201A2E3B0E0E2E3F0E0808168
:102960008F7E8C932091A5013091A6018091A301C7
:102970009091A401A901481B590BCA019093A6018B
:102980008093A5018091A5019091A6018A5F904056
:102990009093A6018093A5018091A5019091A60135
:1029A00029E130E0B9010E944D15CB019093B001AF
:1029B0008093AF018091AF019091B00151E08836D2
:1029C000950730F087E691E09093B0018093AF01D6
:1029D0008091A5019091A6012AEF30E0B9010E94F3
:1029E0004D15CB0190934B0280934A0281E0809376
:1029F0009301DF91CF91FF91EF91BF91AF919F91A3
:102A00008F917F916F915F914F913F912F910F9097
:102A10000FBE0F901F901895FB01DC010D90002058
:102A2000E9F711974150504028F0019000200D9295
:102A3000C9F708951C920895FB019F01E894423064
:102A4000C4F04532B4F44A3029F497FB1EF4909553
:102A500081959F4F642F77270E944D15805D8A33A3
:102A60000CF0895D8193CB010097A1F716F45DE22C
:102A700051931082C9010C943D15DC01FC010190B9
:102A80000020E9F73297AE17BF0730F47C916081E0
:102A9000708331976D93F7CF0895AA1BBB1B51E14B
:102AA00007C0AA1FBB1FA617B70710F0A61BB70BBE
:102AB000881F991F5A95A9F780959095BC01CD0163
:102AC000089597FB092E07260AD077FD04D0E5DF8D
:102AD00006D000201AF4709561957F4F0895F6F79F
:082AE000909581959F4F089528
:102AE800010200000A3100004400002300230054C2
:102AF8006466536365526200516100506000506023
:102B080000516100526200536365546466676869E6
:102B18006A6B6B6A696867555552555552555552D7
:102B2800555552555552555552555552555552555C
:102B3800555255555255555255555255555255554C
:102B4800525555525555525555525555525555553C
:102B5800555555555555550000000000004F020DBC
:022B68000A0061
:00000001FF
